:1000000014C1000042C1000040C100003EC1000018
:100010003CC100003AC1000038C1000036C10000F8
:1000200034C1000032C1000030C100002EC1000008
:100030002CC100002AC1000028C1000026C1000018
:1000400024C1000022C1000020C100001EC1000028
:100050001CC100001AC1000018C100002EC400001D
:1000600014C1000012C1000010C100000EC1000048
:100070000CC100000AC1000008C1000006C1000058
:1000800004C1000002C1000000C10000FEC0000069
:100090005EC40000FAC00000F8C00000F6C0000016
:1000A000F4C00000F2C00000F0C00000EEC000008C
:1000B000ECC00000EAC00000E8C00000E6C000009C
:1000C000E4C00000E2C00000E0C00000DEC00000AC
:1000D000DCC00000DAC00000D8C00000D6C00000BC
:1000E000D4C00000D201D501C401C801CE010C0268
:1000F000D901DD01E301E701EB01F101F501F901AE
:100100000C02FF0103020702000021002400270067
:100110002A002D0030003300010100000401070116
:100120000A0100002200250028002B002E003100CB
:10013000340002010000050108010B01000020004D
:100140002300260029002C002F00320000010000AF
:10015000030106010901050505050705080808084A
:10016000020202020A0A080804040404010101014F
:10017000010101010303030303030303040707074A
:100180000C0C0C0C0C0C0C0C0202020206060606EF
:10019000060606060B0B0B0B0B0B0B0B01021020BC
:1001A00020080810204010204080020102010804AD
:1001B0000201010204081020408080402010080441
:1001C000020180040201804020100804020108049A
:1001D00002010102040810204080010204081020DE
:1001E000408000000A0B02090C0D0E0807030401F1
:1001F00000000000000000000000000000000000FF
:1002000000000000000000000000000000001211CB
:1002100010000000000000000000000000000000CE
:100220000000000000000000B90B11241FBECFEF3A
:10023000D1E2DEBFCDBF00E00CBF25E0A2E7B3E016
:1002400001C01D92AF33B207E1F713E0A0E0B2E0C6
:10025000E4EAFAE100E00BBF02C007900D92A2377A
:10026000B107D9F711E0C5E1D1E000E006C0219760
:100270000109802FFE010E941B0CC431D10780E0D0
:100280000807A9F740D50C94500DBACE8F7799275F
:100290009C0140E050E02115310541F061E0462726
:1002A000B9016150710926233723F5CF452B09F099
:1002B00080680895E1E1F4E020E030E04081411100
:1002C0001DC079E0729FA001739F500D1124FA01A7
:1002D000E950FC4F628FFC0180E090E070E08617EF
:1002E000970754F42191DC01A40FB51FA950BC4F0E
:1002F0005B962C930196F3CF81E008952F5F3F4FDB
:10030000399620313105D1F680E00895CF93DF93FF
:1003100000D01F92CDB7DEB7E82FF0E0282F237072
:10032000220F962F9970292B32E53983F595E795A1
:10033000F595E795EA83922F90689B83E3279E27A4
:100340009C8320E030E0232B39F0462F41704F5F33
:10035000682F80E00E94000064E0CE010196AADFD1
:100360000F900F900F900F90DF91CF91089590E034
:10037000FC013197E231F10508F04EC08827EE58B4
:10038000FF4F8F4F0C941B0C809180008F7703C020
:10039000809180008F7D80938000089580918000FF
:1003A000877FF9CF84B58F7702C084B58F7D84BDF8
:1003B00008958091B0008F7703C08091B0008F7D49
:1003C0008093B0000895809190008F7707C080914E
:1003D00090008F7D03C080919000877F8093900074
:1003E00008958091A0008F7707C08091A0008F7D35
:1003F00003C08091A000877F8093A0000895809122
:1004000020018F7707C0809120018F7D03C08091EC
:100410002001877F809320010895CF93DF93282FB9
:1004200030E0F901EE51FE4F8491F901E456FE4FA0
:10043000D491F901EA5AFE4FC491CC2389F081117D
:1004400096DFEC2FF0E0EE0FFF1FE45CFE4FA5916E
:10045000B491EC91ED2381E090E021F480E002C0C2
:1004600080E090E0DF91CF9108951F93CF93DF93C9
:10047000282F30E0F901EE51FE4F8491F901E45646
:10048000FE4FD491F901EA5AFE4FC491CC23C1F03A
:10049000162F81116CDFEC2FF0E0EE0FFF1FEE5DE9
:1004A000FE4FA591B4918FB7F894111105C09C919E
:1004B000ED2FE095E92302C0EC91ED2BEC938FBF7B
:1004C000DF91CF911F910895CF938230E9F070F4BE
:1004D0008823A9F0813049F5C0917203C827C093E1
:1004E000720360E08CE0C1DF6C2F12C0803291F0AB
:1004F000C09172038F3F99F08430B9F418C060E066
:100500008CE0B3DF61E004C061E08CE0AEDF60E06E
:100510008DE016C060E08DE0A8DF61E010C081E0F2
:10052000C827C09372036C2F07C0C091720381E08B
:10053000C827C093720360E08DE097DF6C2F8CE0DA
:10054000CF9193CFCF93DF9390E0FC01E456FE4F21
:100550002491FC01EA5AFE4F8491882361F190E0D6
:10056000880F991FFC01E85FFE4FC591D491FC01F3
:10057000EE5DFE4FA591B491611109C09FB7F8944B
:100580008881209582238883EC912E230BC06230D2
:1005900061F49FB7F8943881822F809583238883F4
:1005A000EC912E2B2C939FBF06C08FB7F894E88157
:1005B0002E2B28838FBFDF91CF9108953FB7F894FA
:1005C0008091780390917903A0917A03B0917B0395
:1005D00026B5A89B05C02F3F19F00196A11DB11D9E
:1005E0003FBFBA2FA92F982F8827820F911DA11DD9
:1005F000B11DBC01CD0142E0660F771F881F991F16
:100600004A95D1F708958F929F92AF92BF92CF9261
:10061000DF92EF92FF926B017C01D0DF4B015C0116
:10062000C114D104E104F104E9F0C8DFDC01CB011D
:1006300088199909AA09BB09883E9340A105B1050B
:1006400078F321E0C21AD108E108F10888EE880E9B
:1006500083E0981EA11CB11CC114D104E104F10473
:1006600021F7DECFFF90EF90DF90CF90BF90AF905B
:100670009F908F9008952FB7F894609174037091B4
:10068000750380917603909177032FBF0895EF92C1
:10069000FF920F931F93CF93DF931F92CDB7DEB7D7
:1006A0007C018B0161E0FC0182814983DEDEF8017F
:1006B000498150E0CF01801B910B8417950740F4CE
:1006C00081919091C80095FFFCCF8093CE00F2CF2E
:1006D0008091C80086FFFCCF80E48093C800109210
:1006E000C80060E0F70182810F90DF91CF911F91E8
:1006F0000F91FF90EF90B9CE0F931F93CF93DF939D
:10070000EC01862F0AE010E020E030E00A831B8332
:100710002C833D831E821F8291E098871A861B8658
:100720001C861D861E861F86188A198A1C8A1D8AA9
:1007300021E030E03F8B2E8B188E198E1A8E1B8E87
:100740001C8E1D8E1E8E1F8E1AA21BA23DA32CA3D3
:100750006883798362E0F6DE8A819B81AC81BD810A
:100760000097A105B10529F0582F492F3A2F2B2FBB
:1007700004C051E040E030E020E05A874B873C87DE
:100780002D870097A105B10521F481E090E0A0E05C
:10079000B0E0888F998FAA8FBB8FDF91CF911F9187
:1007A0000F9108950F931F93CF93DF93FC0124853E
:1007B0003585232BC9F4EC015EDF0C811D812E8170
:1007C0003F81DC01CB01801B910BA20BB30B088195
:1007D00019812A813B8180179107A207B30720F076
:1007E00081E090E09D878C87DF91CF911F910F91E1
:1007F0000895CF93DF93EC0188810FDE21E0892BF0
:1008000009F420E029878885882311F081E02827D2
:1008100021110FC030DF6C8F7D8F8E8F9F8F1DA2B7
:100820001CA21AA21BA28F8181110BC081E08F83B1
:1008300009C0CE014896B6DF8CA19DA1019709F4AD
:100840001F8280E0DF91CF9108951F93CF93DF93B4
:10085000EC018881E2DD11E0892B09F410E01987B1
:100860008885882311F081E01827112389F003DFA0
:100870006E877F87888B998B1F8A1E8A1C8A1D8AA8
:100880008E81882311F010E00BC081E08E8308C0B8
:10089000CE010A9687DF8E899F890197A1F71E8274
:1008A000812FDF91CF911F91089561E08091F40332
:1008B0002DCD60E08091F40329CD1F920F920FB6E9
:1008C0000F9211242F933F938F939F93AF93BF93D6
:1008D0008091740390917503A0917603B091770392
:1008E0003091730323E0230F2D3720F40196A11DCF
:1008F000B11D05C026E8230F0296A11DB11D20934E
:1009000073038093740390937503A0937603B0935D
:1009100077038091780390917903A0917A03B09145
:100920007B030196A11DB11D8093780390937903F9
:10093000A0937A03B0937B03BF91AF919F918F9166
:100940003F912F910F900FBE0F901F9018951F92FF
:100950000F920FB60F9211240BB60F92EF92FF92E7
:100960000F931F932F933F934F935F936F937F93B7
:100970008F939F93AF93BF93EF93FF93CF93DF93A7
:1009800000D0CDB7DEB700917C0310917D03011537
:10099000110509F4C5C09091C80097FF0FC02091C0
:1009A000C9008091CE009C7149F421FB992790F9F0
:1009B000592F40E09A01282BC90102C08FEF9FEF09
:1009C0008F3F3FEF930709F4ABC0F801E05CFE4FA7
:1009D00010821182128213828F3F910509F008F470
:1009E0008FC0F801118E278130858217930791F40B
:1009F00080E289838A8342E0BE016F5F7F4FC80136
:100A000046DE80E090E0892B09F48AC081EE0E94E6
:100A1000000086C0F801258136818217930709F00E
:100A200052C081E2898384E28A8385E08B8380815E
:100A3000882329F0E35CFE4F80818F3F39F443E047
:100A4000BE016F5F7F4FC80122DE6AC0F801428D90
:100A50004423B1F1838D882329F0B801655E7F4F6F
:100A6000C80115DEF801B396980126553F4F8081E5
:100A7000DF0119978C9380E090E07F014AE1E41A4E
:100A8000F108BF0163527109D701A80FB91F5B9626
:100A90004C91DB01A80FB91F5B964C9301968830EF
:100AA000910591F73996E217F30709F7F801EF5529
:100AB000FF4F108231961192E217F307E1F730C031
:100AC000F801128E2DC08036F1E09F0731F0F80159
:100AD000238134818217930799F4F80112861186D5
:100AE0001486138616861586108A1786128A118A2E
:100AF000148A138A168A158A108E178A21E0218F8C
:100B0000F801218D222361F0218532852F5F3F4F2F
:100B100032872187220F331FE20FF31F92878187CD
:100B20000F900F900F90DF91CF91FF91EF91BF91B8
:100B3000AF919F918F917F916F915F914F913F9175
:100B40002F911F910F91FF90EF900F900BBE0F9080
:100B50000FBE0F901F90189529E0829FC0011124AD
:100B600089509C4FFC01E655FF4F20812F3FE1F457
:100B7000319620812F3FC1F4329620812F3FA1F47E
:100B8000319620812F3F81F4319620812F3F61F4EF
:100B9000319620812F3F41F4319620812F3F21F45F
:100BA000319681E09081911180E00895EF92FF925B
:100BB0000F931F93CF93DF93F82EE62E07EF13E0EA
:100BC000C0E0D0E0F801E655FF4F80818E1104C0EF
:100BD000319680818F1521F08C2FBEDF882359F04C
:100BE0008C2FBADF8823B1F189E08C9F90018D9F13
:100BF000300D112418C02196075F1F4FCF30D1054B
:100C000009F7E9EAF4E090E0C0E08FEF20812817CF
:100C100010F4822FC92F39969F5F9F30B9F789E072
:100C2000C89F9001112429503C4FF901E655FF4F10
:100C3000E0823196F08231968BE08083319610828B
:100C40003196108231961082319610823196108240
:100C5000319610828C2FDF91CF911F910F91FF90D1
:100C6000EF9008958F92AF92CF92EF92FF920F93F1
:100C70001F93CF93DF93182FF62E98DFC82FD0E065
:100C800059E0859F9001112429503C4FF901E4550A
:100C9000FF4F4081329690813196A08031968080BE
:100CA0003196808160E070E0672BB1F0592F5F7161
:100CB000C52E95FBEE24E0F83497242F237043FBD8
:100CC000442740F991E09F938F9300816F2D812FEE
:100CD0000E9400000F900F9089E08C9FF0018D9F83
:100CE000F00D1124E755FB4F80818F3F11F08F5F8E
:100CF0008083DF91CF911F910F91FF90EF90CF9064
:100D0000AF908F900895CF93DF93CDB7DEB7A897BC
:100D10000FB6F894DEBF0FBECDBF789484B5826065
:100D200084BD84B5816084BD85B5826085BD85B58F
:100D3000816085BD80916E00816080936E0010920D
:100D40008100809181008260809381008091810088
:100D50008160809381008091800081608093800019
:100D60008091B10084608093B1008091B000816077
:100D70008093B00080919100826080939100809177
:100D800091008160809391008091900081608093B8
:100D900090008091A10082608093A1008091A100C9
:100DA00081608093A1008091A00081608093A00069
:100DB00080912101826080932101809121018160D5
:100DC0008093210180912001816080932001809196
:100DD0007A00846080937A0080917A0082608093A8
:100DE0007A0080917A00816080937A0080917A0005
:100DF000806880937A001092C100FAE0AF2EF2E092
:100E0000BF2EE12CF12C8E010F5F1F4FA6E29A2E10
:100E1000C090F503D090F603CE0CDF1CF501619174
:100E200071915F01C80168DCF801D601892D01903C
:100E30000D928A95E1F7F6E2EF0EF11C28EEE2162C
:100E400028E0F20629F761E08CE07CDB61E08DE0D0
:100E500079DB61E08CE009DB61E08DE006DB60E2DC
:100E600073E080E090E0CFDB60E08CE0FEDA60E0F1
:100E70008DE0FBDA10923605109235051092370599
:100E8000109238051092390510923A05F4DB609300
:100E90002E0570932F05809330059093310580E0E7
:100EA00090E0892B21F0809135050E9400008AE1B5
:100EB0008093F80382E08093F90361E043DB60E014
:100EC0008091F903D2DAF090F8038F2D90E0DED90B
:100ED00091609093FF038093FE038F2D806490E0D8
:100EE000D5D991609093FD038093FC038F2D80668C
:100EF00090E0CCD991609093FB038093FA03F8942F
:100F00001092CD008FE08093CC001092C8008CE945
:100F10008093C90086E08093CA00789487EF93E0BD
:100F200090937D0380937C0370E0472E70E0572EF2
:100F3000E0E06E2EE0E07E2E1E0135E0230E311C37
:100F40009ADB4B015C018091020490910304892B90
:100F500009F4DAC2809110048111D6C2809135055E
:100F600090913605892B61F441E050E050933605AD
:100F7000409335054114510419F081E00E940000AE
:100F80008091020490910304803651E0950709F0A6
:100F90005AC0209100043091010480910404909182
:100FA000050424303105C1F581369105A9F58091FC
:100FB0000604909107048130910561F48091080442
:100FC000909109048036910509F07DC21092340594
:100FD00080E078C2009751F4809108049091090450
:100FE0008136910509F06FC282E02AC088309105F0
:100FF00031F484E08093340582E066DA8DC0029794
:1010000009F061C28091080490910904833691052A
:1010100009F059C280E214C08138910509F053C229
:101020008091060490910704892B09F04CC28091AD
:101030000804909109048138910509F044C281E0C7
:10104000809334053FC22091FA033091FB0382174D
:10105000930709F038C22091000430910104233035
:10106000310508F430C28091040490910504833660
:10107000910509F498C050F48136910509F44FC0E8
:10108000C0F48234910509F4E3C11DC2813E91058B
:1010900009F481C028F4833A910509F40EC213C201
:1010A000833E910509F453C1843E910509F4A8C01B
:1010B0000AC28091060490910704829709F003C246
:1010C0002530310508F4FFC18091F70381110AC072
:1010D00081E289838A831B8263E0C801EBD881E0C7
:1010E0008093F703109234058091080490910904CD
:1010F000009791F080FF03C021E02093340581FF29
:1011000003C022E02093340583FF03C020E2209334
:10111000340586FD1092F70380913405D3C1233046
:10112000310509F4D0C180910604909107044397DA
:1011300031F46114710419F082E00E940000809182
:101140000604909107044F9731F46114710419F06B
:1011500081E00E940000809106049091070441976D
:1011600031F46114710419F080E00E940000809154
:10117000060490910704429731F46114710419F048
:1011800083E00E940000809106049091070480385B
:10119000910509F098C16114710409F494C181EEBC
:1011A0000E94000090C180910604909107048197ED
:1011B00069F42530310550F080E090E0892B31F062
:1011C00060910A04809108040E9400008091060446
:1011D000909107048B7F409709F075C180910004BE
:1011E00090910104059708F46EC180910804609104
:1011F0000A04E0E0F0E0309709F465C1199563C195
:101200002730310508F45FC1E0902805F0902905EA
:10121000E114F10409F457C1109229051092280530
:1012200040910604242F277F243009F423E0809185
:10123000080490910904F82FFF77DF2E8078992712
:1012400030910A04C0900C0443FD2860892B19F0EA
:10125000932F906202C0932F9F7D6E2D8F2D28A714
:101260009FA3A4DC482F50E039E0839FF0011124B4
:10127000ED55FB4F808128A59FA1821719F020838F
:1012800021E001C020E089E0849FF001859FF00DFE
:101290001124EC55FB4F80818D1511F0D08221E097
:1012A00089E0849FF001859FF00D1124EB55FB4FE1
:1012B0008081891711F0908302C0222371F089E0A8
:1012C000849FF001859FF00D1124E755FB4F80812D
:1012D0008F3F11F08F5F808321E06E2D8F2D28A727
:1012E00065DC49E0849FC001112489509C4FFC01BA
:1012F000E155FF4F308128A53C1541F0C08233965F
:1013000080818F3F29F08F5F808302C0222319F0F4
:101310006E2D8F2DA7DCD110D6C082E98983FA8289
:10132000EB828F258E258C8364E0C8010E945A01D0
:101330006E2D8F2D3BDC59E0859FC0011124FC01EF
:10134000EC55FB4F10826E2D8F2D8CDCBCC0809134
:101350000604909107048235910509F051C02630AA
:10136000310508F44DC0E0902C05F0902D05E114F6
:10137000F10409F445C010922D0510922C054091FE
:10138000080420910A046E2D8F2D28A74FA30EDC90
:10139000682F70E099E0899FF0011124E955FB4F17
:1013A00080814FA128A5841719F0408381E001C0F6
:1013B00080E099E0969FF001979FF00D1124E85589
:1013C000FB4F9081921711F0208302C08823C1F057
:1013D00089E0869FF001879FF00D1124E755FB4FB0
:1013E00080818F3F11F08F5F808380E090E0892BB8
:1013F00021F06E2D8F2D0E9400006E2D8F2D32DC7E
:1014000080910604909107048034910509F05BC037
:101410008091000490910104069708F454C06091F3
:101420000A0480910804C2DBE9E08E9FC001112408
:1014300089509C4FFC01E455FF4F20812860208398
:10144000369680818F3F09F43EC08F5F80833BC01A
:1014500023303105C1F1E0900604F0900704EE0C52
:10146000FF1CEE0CFF1C8091080490910904482F8A
:1014700043709C013695279536952795F22FF3708A
:10148000DF2E64E0969587956A95E1F780FF03C0AB
:1014900022E0E20EF11C80E090E0892BA1F06E2D9D
:1014A0008F2D0E94000061E06E0D9FEFE91AF90A8E
:1014B0004D2D8F2D0E94000006C02330310519F0FC
:1014C0008091060401D81092010410920004109239
:1014D0000304109202041092050410920404109266
:1014E0000704109206041092090410920804109246
:1014F0000B0410920A0410920D0410920C04109226
:101500000F0410920E0435C0809137059091380574
:10151000A0913905B0913A050196A11DB11D8093A6
:10152000370590933805A0933905B0933A05853077
:101530009942A105B105ECF01092F703109237051E
:10154000109238051092390510923A0581E02091E9
:10155000350530913605232B09F080E0282F30E047
:1015600030933605209335054114510411F00E9443
:10157000000080912E0590912F05A0913005B0912B
:101580003105A5019401281B390B4A0B5B0B293C43
:1015900031054105510598F180922E0590922F0555
:1015A000A0923005B092310520912805309129058F
:1015B0002115310521F180912A0590912B05019685
:1015C00090932B0580932A050A97CCF085E0F801CB
:1015D00011928A95E9F783EE89833B832C8380E01F
:1015E000F80191918927E215F305D9F78D8365E01C
:1015F000C8010E945A0110922B0510922A0582E818
:10160000C82E82E0D82E9AEF892E92E0992E2EEBEA
:10161000A22E22E0B22EE12CF12C8091F5039091C4
:10162000F6038E0D9F1D11D98823D1F1F40180811D
:1016300081508093F403F50190819923C9F068E00B
:101640000E948601F6018081882339F068EC70E001
:1016500080E090E00E94030309C08091F50390911F
:10166000F6038E0D9F1DC5D88823B9F322D918C063
:1016700069E00E948601F6018081882339F068ECD8
:1016800070E080E090E00E94030309C08091F503C0
:101690009091F6038E0D9F1DACD88823B9F305D920
:1016A000F6E2EF0EF11C2FEFC21AD20A32E0830EDF
:1016B000911C4FEFA41AB40A58EEE51658E0F5064F
:1016C00009F0ABCF8EEC93E0C0D8882351F081E2D3
:1016D000898381E88A8380EA8B8363E0C8010E9462
:1016E0005A0188EA93E0B1D8882351F081E28983D6
:1016F00080E88A8381EA8B8363E0C8010E945A01F3
:1017000082E893E0A2D8882339F080E889838A832D
:1017100062E0C8010E945A010E943B03C0907E0310
:10172000D0907F03E0908003F09081039B01AC0197
:101730002C193D094E095F0969017A0135EFC3167D
:1017400031E0D306E104F10460F060937E0370930E
:101750007F038093800390938103809134050E94DE
:10176000640240E050E0452B09F4EACB0E940000FF
:10177000E7CB88EE98E067D09093F6038093F5036B
:101780008FEF8093340580E090E0FC01E950FC4F3E
:10179000128E20E030E0DF01A20FB31F5B961C9297
:1017A0002F5F3F4F28303105B1F7099680399105F9
:1017B00061F71092F70387EF93E02FEFFC01E655F6
:1017C000FF4F2083319620833196208331962083EA
:1017D0003196208331962083319620833196208361
:1017E00031961082099634E08E37930739F71092BC
:1017F00029051092280510922B0510922A051092A7
:101800002D0510922C05109233051092320510927E
:1018100010046AE070E08EEC93E00E947C036BE0C1
:1018200070E088EA93E00E947C0369E070E082E85F
:1018300093E00C947C03EE0FFF1F881F8BBF079073
:10184000F691E02D1994CF93DF938230910510F437
:1018500082E090E0E0913D05F0913E0520E030E02F
:10186000C0E0D0E0309711F140815181481759070D
:10187000C0F04817590761F482819381209719F0CD
:101880009B838A832BC090933E0580933D0526C0A1
:101890002115310519F04217530718F49A01BE01BA
:1018A000DF01EF010280F381E02DDCCF211531054E
:1018B00009F1281B390B2430310590F412968D91D3
:1018C0009C9113976115710521F0FB01938382832D
:1018D00004C090933E0580933D05FD01329644C0BF
:1018E000FD01E20FF31F81939193225031092D9353
:1018F0003C933AC020913B0530913C05232B41F4A9
:10190000209102023091030230933C0520933B0565
:1019100020910002309101022115310541F42DB7CB
:101920003EB74091040250910502241B350BE09113
:101930003B05F0913C05E217F307A0F42E1B3F0B8B
:101940002817390778F0AC014E5F5F4F2417350731
:1019500048F04E0F5F1F50933C0540933B05819329
:10196000919302C0E0E0F0E0CF01DF91CF910895C4
:101970000F931F93CF93DF93009709F48CC0FC0162
:1019800032971382128200913D0510913E05011598
:10199000110581F420813181820F931F20913B0535
:1019A00030913C052817390779F5F0933C05E09311
:1019B0003B0571C0D80140E050E0AE17BF0750F4BE
:1019C00012962D913C911397AD012115310509F126
:1019D000D901F3CF9D01DA013383228360817181C4
:1019E000860F971F8217930769F4EC0128813981CC
:1019F000260F371F2E5F3F4F318320838A819B81C3
:101A000093838283452B29F4F0933E05E0933D05B3
:101A100042C01396FC93EE931297ED0149915991B0
:101A20009E01240F351FE217F30771F48081918125
:101A3000840F951F029611969C938E9382819381B9
:101A400013969C938E931297E0E0F0E0D8011296E3
:101A50008D919C911397009719F0F8018C01F6CFA6
:101A60008D919C9198012E5F3F4F820F931F209183
:101A70003B0530913C052817390769F4309729F464
:101A800010923E0510923D0502C0138212821093FF
:101A90003C0500933B05DF91CF911F910F91089575
:041AA000F894FFCFE8
:101AA40000003F05800001000000360037003800C8
:101AB40039003A003B003C003D003E003F0040003E
:101AC40041004200430044004500110010000F0093
:101AD4000E000300040005000600070008001600BD
:101AE40018001A001C001E002000240022002C00F4
:101AF4002A00280026002E00300032003400350071
:101B0400330031002F002D002B0029002700250071
:101B1400230021001F001D001B00190017001500E1
:101B2400140001010101010101010101010101018F
:101B34000101010101010101010101010101010191
:101B44000101010101010101010101010101010181
:101B54000101010101010101010100000000010076
:101B64000100010001000100010001000100010069
:101B74000100010001000100010001000100010059
:101B84000100010001000100010001000100010049
:101B94000100010001000100010001000100020038
:101BA4000200030003000400040005000500060011
:101BB40006000700070008000800090009000A00E1
:101BC4000A000B000B000C000C000D000D000E00B1
:101BD4000E000F000F001000100011001100120081
:101BE4001200130013001400140015001500160051
:101BF40016001700170018001800190019001A0021
:101C04001A001B001B001C001C001D001D001E00F0
:021C14001E00B0
:00000001FF
